:020000000528D1
:080008008928FF2383169000F4
:1000100083128501A20107309900831668309F0082
:1000200000309500383085008F30810083127520B4
:100030009720972064007520851E2210851A2214AF
:10004000851DA2108519A21422182C28A2182C286C
:100050002211A2112212A212221C3428A218342822
:10006000A21A34282215A21122183E28A21C3E28CA
:10007000221A3E282211A2152216A216221C44285A
:10008000A21C44282211A211503020020318492832
:1000900005112008663C03184E2805155130200232
:1000A0000318532822132008A33C03185A282217A8
:1000B0002216A216221F61282211A21105108510F6
:1000C0007328221D6928A219692885100514221693
:1000D0007328A21D71282219712805108514A216F3
:1000E0007328051085108A201A288D309F00810101
:1000F000811E78289F149F187B281E08A100831654
:100100001E08A0008312210803190800FF30A00078
:10011000080009006A30A300000000000000000091
:10012000A30B8C28000000000000000008004130F4
:10013000A4008A208A208A208A208A208A208A2075
:0E0140008A208A208A208A20A40B9928080091
:02400E000C3F65
:00000001FF
